:030000000211F7F3
:03000B000200C12F
:03002B000203CB02
:03005B0002051D7E
:0300730002051370
:1000800002030406080C10182030406080020304AC
:1000900006080C101820304080FF0406080C1018C9
:1000A0002030406080A0C000000001010003020277
:1000B000010D0D040506020D0505050D06030502DB
:1000C00002C2AFC0D0C0E0205A0D302F02E473301E
:1000D000600280F90203B7306306C293C295C297EB
:1000E00085258AC25AE525F4700221AA056130608F
:1000F00013206A19758B00D0E0D0D0C293C295C28C
:1001000097D2AF32C293C295C29702019AD26EC201
:100110006FE565601CC3E5611495654014C26ED23D
:100120006FC3E5619564500302019A756100020195
:100130009A206C14C293C295C297740AD5E0FDD27E
:1001400092D294D29602019AC293C295C297E53D8B
:1001500020E22520E10D207502D292307502D29660
:1001600002019A20E005D29402019A207502D296EB
:10017000307502D29202019A20E11520E00D20751F
:1001800002D292307502D29602019AD29402019A5A
:10019000207502D296307502D292758B00D0E0D0D5
:1001A000D0C293C295C297D2AF32D0E0D0D0D2AFF6
:1001B0003261B7E525600A207502D293307502D20C
:1001C00097C29561B7E5256002D295207502C29766
:1001D000307502C29361B7E525600A207502D29797
:1001E000307502D293207502C293307502C29761B6
:1001F000B7207502C292307502C296E525600A20CA
:100200007502D293307502D297207502C29630756E
:1002100002C292C29561B7207502C292307502C2C5
:1002200096207502C296307502C292740AD5E0FD1E
:10023000E525600A207502D293307502D297C295E7
:1002400061B7207502C292307502C296E525600A38
:10025000207502D293307502D297C294C29561B7CD
:10026000207502C292307502C296C294740AD5E01B
:10027000FDE525600A207502D293307502D297C23F
:100280009561B7C294E5256002D295207502C292AD
:10029000307502C296207502C297307502C2936112
:1002A000B7C294207502C292307502C296740AD504
:1002B000E0FDE5256002D295207502C297307502F7
:1002C000C29361B7C294E5256002D295207502C23F
:1002D00096307502C292207502C297307502C293A1
:1002E00061B7C294207502C296307502C292740A38
:1002F000D5E0FDE5256002D295207502C2973075E4
:1003000002C29361B7207502C296307502C292E5AF
:1003100025600A207502D297307502D293C29420CC
:100320007502C293307502C29761B7207502C296FA
:10033000307502C292C294740AD5E0FDE525600AC8
:10034000207502D297307502D293207502C2933085
:100350007502C29761B7207502C296307502C292CB
:10036000E525600A207502D297307502D293207578
:1003700002C292307502C296207502C29330750295
:10038000C29761B7207502C296307502C29220757D
:1003900002C292307502C296740AD5E0FDE525606E
:1003A0000A207502D297307502D293207502C2934B
:1003B000307502C29761B7E525F4F58A758B007533
:1003C0006000D25AD0E0D0D0D2AF32C2AFC0D0C0DD
:1003D000E0D2D3C2CEE528600A741F552E604915BD
:1003E00028812878007900E580307601F430E30236
:1003F00078FF53DACF20760343DA2030760343DAEE
:1004000010C2D8C269E580307601F430E30279FF8A
:10041000C3E89970CE305903752818741F552E60A3
:10042000037528188858D268E52960041529813B8E
:10043000741F552E600543DA01C2D820680281CDB1
:10044000E558F8C268741F552E60367982B70431BA
:10045000C3E894F0400374F0F8E8C4540F28F87926
:1004600084B703028181C313C3138721200802C309
:0E04700013200A06C3C898F8818128F85003AB
:10047E0074FFF8C3E8955F5003E55FF8E52C54066A
:10048E00703D882230630AC3E522955C4003855C8B
:10049E00227882B60429C3E5229524401278A096CC
:1004AE00400DE52426F52450097524FF0204C0856D
:1004BE002224852425C3E524955C4003855C2520F4
:1004CE00CF09D0E0D0D0C2D3D2AF32C2CF7801E5BF
:1004DE00286008741F552E70021528C3E558940124
:1004EE004005755B0081FCE55B046002055BE55D24
:1004FE00C3240A5005755DFFA10AF55DD0E0D0D08A
:10050E00C2D3D2AF32C2AF53917FC258D2AF32C232
:10051E00AFC0D0C0E0C0F0D2D3A8FBA9FCC2D83087
:10052E006902A18053DACF20760343DA10307603C6
:10053E0043DA20D269E580307601F420E302A1543B
:10054E0088268927E12053DACF20760343DA20303C
:10055E00760343DA10C2D8C269741F552E7002E1B9
:10056E00067800E580307601F430E302E106885823
:10057E00E10653DACF20760343DA2030760343DAEE
:10058E0010C269205902C13A53DACF20760343DAFA
:10059E001030760343DA20C2D8D26988538954C307
:1005AE00E89551F8E99552F9E4FB7AFAC3E894C854
:1005BE00E994005008E4D2E4FB7A0AC10DC3E89432
:1005CE0068E994015008E4D2E3FB7A0FC10DC3E849
:1005DE0094D0E994025008E4D2E2FB7A1EC10DC316
:1005EE00E894A0E994055008E4D2E1FB7A3CC10DF1
:1005FE00C3E89498E994085006E4D2E0FB7A78C3F5
:10060E00E89555FCE99556FD30E708ECF42401FC1D
:10061E00EDF4FD7557007008C3EC9A500375570141
:10062E0088558956A853A95488518952C3E89526EE
:10063E00F8E99527F9307402C1D9307302C1D93067
:10064E007202C1D2E9C313F9E813F8307102C1D2B4
:10065E00E9C313F9E813F8307002C1D2E9C313FDF0
:10066E00E813FC205918C3EC941CED9402400302CD
:10067E000706ED7009C3EC94C850030207207400FE
:10068E002077037896E624FAFEE43400FFC3EC9E4E
:10069E00FCED9FFD500678007900C1D9C3EC94FFA4
:1006AE00ED9400400678FF7900C1D9EC856CF0A47A
:1006BE00C5F0A2F733F8790040030206F578FF790A
:1006CE00000206F5E9C313F9E813F830740EE96079
:1006DE000278FFC3E81338F8E43400F9C3E894FF56
:1006EE00E99400400278FF8858D268205902E1064A
:1006FE00741FF4552E4BF52E752818741F552E7039
:10070E000375280A305902E120741F552E600353D9
:10071E00DAFE752906741F552E700375290AD0F05E
:10072E00D0E0D0D0C2D3D2AF327901E14F7903E11C
:10073E004F790AE14F791EE14F7964E14F79C8E1B3
:10074E004F7817E4D5E0FDD8FAD9F6227A147B78E3
:10075E000207767A107B8C0207767A0D7BB402073D
:10076E00767A0B7BC8020776AC257525017902B225
:10077E0075E4C294D5E0FDE5256002D295D5E0FD85
:10078E00C295D5E0FDD294D5E0FDE525600A207531
:10079E0002D293307502D297E56DD5E0FD20750239
:1007AE00C293307502C2977496D5E0FDD9C1EAF8AE
:1007BE00D5E0FDD8FBDBB1C2948C2522C37C007D35
:1007CE000075F00005F0EA33FAEB33FB50F6EB134D
:1007DE00FBEA13FAC3E9FFE8FEE89AF8E99BF95041
:1007EE0004EFF9EEF8B3EC33FCED33FDD5F0DFEDAD
:1007FE00F9ECF822E889F08A20D2D4F8A9F07B002F
:10080E0030F70B7BFFF42401F8E9F43400F9E885A6
:10081E0020F0A4ADF0F8E98520F0A4AFF0FEED2EA7
:10082E00F974003FFA7C04C3EA13FAE913F9E813EA
:10083E00F8DCF48BF030F70AE8F42401F8E9F4342C
:10084E0000F9E889F0C2D4F8A9F0227882B6040340
:10085E000208B6C3E5589401400302087E8522249F
:0D086E00E4F53FF540F541F542F543F5484E
:10087B000208B67882E6FC754801E522F523783844
:10088B0079C7AA3BAB3CC3EB13FBEA13FAEC14603E
:10089B0013C3EB13FBEA13FAEC14146007C3EB134B
:1008AB00FBEA13FA1207CA883F894022E5486034F5
:1008BB00C3E53F9523F8E5409400F9500CC3E89449
:1008CB0080E994FF40160208EBC3E8947FE994009B
:1008DB0050030208EB787F79000208EB788079FFF0
:1008EB008844894522E5486058E5442541F8E545AB
:1008FB003542F9854520E4300701F43543FA30E7FA
:10090B0009C3EA94F0401502092DC3EA940F500372
:10091B0002092D78FF79FF7A0F02092D78007900F3
:10092B007AF0C3E524955C5006E52460092146E581
:10093B004520E70D2146E54530E706884189428A87
:10094B004322E54870030209B0789EE6FAC3E544FA
:10095B0033F8E54533F91102E930E70BC3E894802E
:10096B00E994FF40132187C3E8947FE99400500278
:10097B002187787F79002187788079FFE820E71538
:10098B00C3E52398F84009C3E8940140030209AE7C
:10099B0078010209AEE8F424012523F8400302098B
:1009AB00AE78FF884622E5487003020A12789FE66C
:1009BB00FAA842A9431102E930E70CC3E89401E914
:1009CB0094FF40160209E9C3E894FFE99400500331
:1009DB000209E978FF79000209E9780179FFE9203A
:1009EB00E715C3E54698F84009C3E89401400302B4
:1009FB000A107800020A10E8F424012546F8400397
:100A0B00020A1078FF8824227883E6F520120F68FB
:100A1B0075E890E5E820ECF0A8BDA9BE12100075B2
:100A2B006830756900C3740013FD743013FC7430A7
:100A3B002CFC74003DFDECFAEDFBC3E89AE99B40FE
:100A4B0014E5682430F568E5693400F569EA2CFA99
:100A5B00EB3DFB80E5AE68AF69C3E56913F9E5686B
:100A6B0013F8C3E913F9E813F8E56828F566E569A7
:100A7B0039F5677A03C3E913F9E813F8DAF7AA2013
:100A8B001A7009756800756900020AA71AEA6008EE
:100A9B00EE28FEEF39FFDAF88E688F692275E89041
:100AAB00227883E6FFE5E820ECF7A8BDA9BE056A2E
:100ABB00C3E56A94084052756A00E97007E56B60FC
:100ACB001B020ADBC3E8956B6010E56B5006600CEC
:100ADB0014020AE70460F9020AE7E56BF56BC394AD
:100AEB00A8F84021755CC0C3E89405F84017755C05
:100AFB0080C3E89405F8400D755C40C3E89405F895
:100B0B004003755C0075BB0122EFC39401601BC3EE
:100B1B00E894FFE994035012C3E89568E99569508E
:100B2B0009E55C600C155C020B3CE55CF4600205AE
:100B3B005CA85CC3E524985002A8248825C3E5254E
:100B4B00955D400B855D25E55DF46003855D5CC3BC
:100B5B00E56AB4070375BB1E22306102783230623E
:100B6B00027878E52C5406601FE879A187F0A4C5BC
:100B7B00F0A2F733F8C3E8955C4002A85C882288A2
:100B8B00248825306102885E22788FE6FFC3EF94BC
:100B9B00055018C3EF94045020C3EF94035028C39F
:100BAB00EF94025030C3EF940150387533A0753475
:100BBB000F75353C75360561FC7533C07534127590
:100BCB00354075360661FC7533707534177535D045
:100BDB0075360761FC75334C75341D7535C4753628
:100BEB000961FC7533287534237535B875360B617F
:100BFB00FC85334F853450753B00753C0822A84F5C
:100C0B00A950020C14A849A94A759100C3E498F5A0
:100C1B0094E499F595759104D25875C820A8CCA980
:100C2B00CD75C824AA39AB3A8839893AC3E89AF802
:100C3B00E99BF9AA3BAB3CC3EB13FDEA13FCC3EDF9
:100C4B0013FDEC13FCC3EA9CFAEB9DFBEA28FAEBD1
:100C5B0039FB8A3B8B3C400122753BFF753CFF22E5
:0F0C6B00305802816B759100C3E4954BF594E40A
:100C7A00954CF595759104D258227892E6FF7E102C
:100C8A00305B027F053063047F037E00A93CA83BEA
:100C9A007A04C3E913F9E813F8DAF7C3E89EF8E926
:100CAA009400F94009C3E89402E9940050047802D8
:100CBA00E4F9E9FBE8FAC3E913FDE813FCC3EF948E
:100CCA0003602EEF20E00DE82CF8E93DF9ECFAED8F
:100CDA00FB020CE8E828F8E939F97A02E4FBC3EFE9
:100CEA009403400D8A4D8B4E8849894A8C4B8D4C12
:100CFA0022884D894E8A498B4A8C4B8D4C2230581A
:100D0A0002A108759100C3E4953BF594E4953CF57E
:100D1A0095759104D25822753E00752000020D3057
:100D2A00753E00752040D2AF053E20580122759DC0
:100D3A0000759C00E53CC313C313F8086036306A9B
:100D4A0006C313C313F808C3E8940A4002780A30AA
:100D5A006D08C3E8940440027804C3E53C94084053
:100D6A0013759D02759C02C3E53C94104006759D5F
:100D7A0003759C03205803D2AF22791E206D027995
:100D8A000AD2AF0000C2AF205A0A793C206D02791C
:100D9A0014306FE03063027978C3E58B9940D5E56A
:100DAA009E7005E59B020DB4E59AF45440B5200205
:100DBA00A130D8C0D2AF22C25B789CE6146007E5A6
:100DCA003E147002D25B30630B0538205810753818
:100DDA0000020DE82058071581158102175822755F
:100DEA009100C3E4954DF594E4954EF595759104FB
:100DFA00D25822AE25305B4F78A3E6FFBF010BD253
:100E0A005C752500C293C295C2979170305C0375D8
:100E1A002500305802C116BF020BD25C752500C2EC
:100E2A0093C295C29778A2B6010D9170305C037592
:100E3A002500305802C136BF030BD25C752500C2AB
:100E4A0093C295C297B1E9305C0375250030580208
:100E5A00C151305B04C25C8E2522C2AFC294206AA3
:100E6A0003020E86900305206C12306E0F20750265
:100E7A00C296307502C292740AD5E0FD207502D27C
:100E8A0092307502D296759F33759E00753D02D2D7
:100E9A00AF22C2AF206A03020EBE9002C4306E17A0
:100EAA00C294207502C296307502C292740AD5E0C5
:100EBA00FD020EC19001C5207502C297307502C2AB
:100ECA0093305A06E5256002D295207503759E2354
:100EDA00307503759E22753D03D2AF22C2AF2075CD
:100EEA0002C292307502C296206A03020F0890026B
:100EFA0083206C0A306E07C294740AD5E0FD20750F
:100F0A0002D296307502D292207503759E223075F0
:100F1A0003759E23753D04D2AF22C2AF206A030235
:100F2A000F46900242306E17207502C29230750247
:100F3A00C296C294740AD5E0FD020F499001B3C269
:100F4A0095305A0EE525600A207502D29330750253
:100F5A00D297759F33759E00753D05D2AF22C2AFF9
:100F6A00207502C296307502C292206A03020F925D
:100F7A009001F1206C12306E0F207502C29230750A
:100F8A0002C296740AD5E0FDD294207503759E2399
:100F9A00307503759E22753D06D2AF22C2AF206A14
:100FAA0003020FD0900356306E1F207502C2923092
:100FBA007502C296207502C296307502C292740AF0
:100FCA00D5E0FD020FD39001D7207502C293307588
:100FDA0002C297305A0EE525600A207502D2973070
:100FEA007502D293207503759E22307503759E2370
:100FFA00753D01D2AF229001B1C293C295C297C288
:10100A0092C294C29622C3E54F9535E55095365063
:10101A0001227890E6FFC3EF94055018C3EF9404B9
:10102A00501BC3EF9403501EC3EF94025021C3EF29
:10103A0094015024C3E54F943CF802106BC3E54F6A
:10104A009428F802106BC3E54F941AF802106BC388
:10105A00E54F9412F802106BC3E54F940AF8021098
:0E106A006BE5509400F9884F895022305803EE
:101078000210752278807607788176077882760163
:10108800788476037883760178867607788F760178
:10109800789076057895760278927603789B760D27
:1010A8007893760678877601789C76027888760138
:1010B8007889760178857600788C7601788D760047
:1010C800788E76B478967625789776D078987678EC
:1010D800789976C8789A7604789D7600227893E68F
:1010E800FF756409756501C3BF02097564057565F7
:1010F8000102112AC3BF030975640575650202114F
:101108002AC3BF040975640575650302112AC3BFA4
:101118000506756409756507C3BF0606756400751D
:1011280065007887E6FFC26CC3BF0302D26CC26B4E
:10113800C3BF0402D26BC26A7418552D6002D26A0A
:10114800C26E6002D26ED26F6002C26FC2757888BA
:10115800E630E102D275C2767889E630E102D276CD
:10116800C3EF94026008758E01D26D02117B758EF3
:1011780000C26D227880E61490008093789EF678FD
:1011880081E61490008093789FF6110022789BE600
:101198001490008D9378A0F61100227886E61490BA
:1011A800009A9378A1F6110022789CE6149000A783
:1011B8009378A2F6789CE6149000AC9378A3F61185
:1011C8000022227896E6FA7897E6FB3077047A00D0
:1011D8007BFFC3EB9AFCC3948250027C82756C003F
:1011E800056CEC856CF0A4C3E5F0948040F222C253
:1011F800D353D9BF7581C043FF8012073775EF02FB
:1012080043B203E5B324044002F5B37580FF75A427
:101218000075F1FE75D4F775900275A5FC75F2FCA2
:1012280075D50075A0FD75A60275F30275D6007513
:10123800B0FF75A70175F4FF75E2411100E4F8F6F7
:10124800D8FD117C12178611E5317C319531A33117
:10125800B131CA31CB7898866D110075885075897F
:101268000275C82475910475D84012074B12075AA5
:101278001207431207611207431207681207431245
:101288001CE512074B12074B12074775A82275B8C1
:101298000275E69075F610759B80759D03759A80AA
:1012A800759C0375D10E75BC5875BB0175BA1F7551
:1012B800E880120737D2AF120A1343DA01C2D8C244
:1012C8006912074B753001D2597A05E55770027AD1
:1012D8000512073BE558C3940240EEE52E541F85DE
:1012E8005A59F55AB559E2DAE2C25953DACF20769B
:1012F8000343DA2030760343DA10C2D8C2691207F2
:101308004712073B7802741F552E70027800C3E518
:10131800589840EDC2AF12075A12075A12075AD20C
:10132800AF12074B75470012073B788CE6C3940150
:1013380050030213F8E530C3940150030213F87404
:101348001F552E6035C3E55894FF50030213F8C2A9
:10135800AF12076FD2AF120747C3E558940150EF99
:10136800C2AF12075A12073F12075AD2AF120747E5
:10137800C3E55894FF40E9021D6A7F05D27731CB57
:10138800120747C2AFC27731CBC3E558947FD2AFBB
:101398004068C2AF12076FD2AFDFE1C3E5589405CA
:1013A8007897F612074B121835121CED7F0AD27780
:1013B80031CB120747C2AFC27731CBC3E558947F10
:1013C800D2AF50E8C2AF12075A12073F12075AD2DB
:1013D800AFDFDBE55824057896F612074B1218356F
:1013E800121D1C120747C3E55894FF40F6021D6AF8
:1013F800C3E55895474003855847120747C3E55842
:1014080094014002612FC2AF12076F12076F1207D3
:101418006FD2AF12074B753000E4F531F532053164
:10142800E531F470360532789AE678281460127837
:101438005014600D78A014600878F01460037532B9
:1014480000C3E53298401415327899866DC2AF1200
:10145800076FD2AF7898866D12074712073BE528C9
:0F1468007008741F552E700241CFC3E5589406CB
:1014770040AD120747E52870030212CF1100E4F5CB
:1014870022F523F524F525755CFF7885865FF53F02
:10149700F540F541F542F543F56AF548F52BF52C8E
:1014A700F55B120B94756A0875BB1E120737120A93
:1014B700A8E5E820ECFBA8BDA9BEE97001F8886B98
:1014C700120AAC756A0875BB1E7895E630E0030210
:1014D70015157887E6FE760211E57887EEF6D26174
:1014E700C2AF120B6485225C85225DD2AFC26175E3
:1014F7002500756200756301D260D26375380012EA
:101507000F68120FA6120C10120B9402163E788762
:10151700E6FE76037893E6FD760511E57887EEF625
:101527007893EDF6D260D261D26E120F68120FA6D1
:10153700120B64120737120E64120737120737129D
:101547000E9C12073B120EE612073B12073B120FC7
:101557002412073F120F6812073B120737C261D2E6
:1015670062120AA8120AAC120B64756A0875BB1ED0
:10157700120FA6120C09120C8411101175120E64A9
:10158700120C09120C8411101175120E9C120C0901
:10159700120C8411101175120EE6120C09120C842C
:1015A70011101175120F24120C09120C841110114D
:1015B70075120F68120C09120C841110C3E54F95B0
:1015C70035E5509536400C1175C3E5589401509197
:1015D7000217581175C2627887E6FE760211E57820
:1015E70087EEF685225C855E5D855E2575620075F2
:1015F7006301D263753800C2AF207502C29230759D
:1016070002C296207502C296307502C292742DD519
:10161700E0FDD2AF120FA6120C10120C6B120C8445
:10162700120D08756A0075BB0102163E11E5120F0F
:10163700A6756A0075BB01120D2A120DC1120DE9BC
:10164700120859120DFD120E64120C10120C6B12B7
:101657000C84120D08120D21120DC1120DE912088A
:10166700B7120DFD120E9C120C10120C6B120C848B
:10167700120D08120D2A120DC1120DE91208F012EF
:101687000DFD120EE6120C10120C6B120C84120DCB
:1016970008120D21120DC1120DE912094D120DFD8F
:1016A700120F24120C10120C6B120C84120D08125C
:1016B7000D2A120DC1120DE91209B1120DFD120FFB
:1016C70068120C10120C6B120C84120D08120D21EB
:1016D700120AA8120DC1120DE9120AAC120DFD1261
:1016E7000FA6120C10120C6B120C84120D0830632B
:1016F7002A855E5C855E5D756200756301C3E538AA
:101707009464400AC263D264753714021722C3E592
:10171700589401400302163E021758306419E53702
:10172700147005C264021633F537C3E558940140B7
:101737000302163E021758C3E55B94FA5013741F51
:10174700552E7004E5286009C3E53C94F05002C1AA
:101757003E11007887E6FE760211E57887EEF6E41B
:10176700F522F523F524F525F55FC2601207371139
:1017770000741F552E7006E528700241CF81219015
:101787001A0D7820121C00E520B4550CA3121C007A
:10179700E520B4AA030217A7117C121835021834E2
:1017A700901A037880121C00A308121C00A30812C9
:1017B7001C00901A067883121C00A308121C00A3B1
:1017C70008A308121C00A308121C00A308121C007F
:1017D700A308121C00A308A308A308121C00A3084F
:1017E700A308121C00A308121C00A308121C00A3C4
:1017F70008A308121C00A308121C00A308A30812C0
:101807001C00A308121C00A308121C00A308121C2A
:1018170000A308121C00A308121C00A308121C0036
:10182700A308121C00A308121C00901A2122C2AFA1
:10183700121C3F121C19901A00740A121C05A3747B
:1018470004121C05A37410121C05901A0378801249
:101857001C04A308121C04A308121C04901A06787F
:0D18670083121C04A308121C04A308A3088C
:10187400121C04A308121C04A308121C04A30812BB
:101884001C04A308A308A308121C04A308A3081299
:101894001C04A308121C04A308121C04A308A30814
:1018A400121C04A308121C04A308A308121C04A3FA
:1018B40008121C04A308121C04A308121C04A30885
:1018C400121C04A308121C04A308121C04A308126B
:1018D4001C04A308121C04121C52121C30901A215E
:0118E40022E1
:101A00000A04100909040103FF0701010155AA0195
:101A1000FFFF0105FF0306FF0225D02850040D0239
:021A200000FFC5
:101A4000235467794B4631323041485623202020B9
:101A500023424C48454C4923463331302320202033
:101A60002020202020202020202020202020202076
:101C0000E493F622E6438F01538FFD75EF0275B71B
:101C1000A575B7F1F0538FFE22438F02438F0175F4
:101C2000EF0275B7A575B7F1901A0DF0538FFC222E
:101C3000901A0D74559105901A0E74AA9105227A86
:101C40003079D07820901A409100E520F709A3DA86
:101C5000F7227A3079D0901A40E7910509A3DAF992
:101C600022AB6EA86FBB01057980021CE2BB0205A6
:101C70007981021CE2BB03057982021CE2BB0405E8
:101C80007984021CE2BB05057983021CE2BB0605D0
:101C90007995021CE2BB07057986021CE2BB0805A8
:101CA000798F021CE2BB09057990021CE2BB0A0590
:101CB0007992021CE2BB0B05799B021CE2BB0C056E
:101CC0007993021CE2BB0D057987021CE2BB0E056D
:101CD000799C021CE2BB0F057988021CE27989021B
:101CE0001CE2E8F7227C0512074BDCFB22C2AF1294
:101CF000075A12076112076812076F12073F12078F
:101D00005A12076112076812076F12073F12075A2B
:101D100012076112076812076FD2AF22C2AF120713
:101D20006F12076812076112075A12073F12076FF6
:101D300012076812076112075A12073F12076F1243
:101D4000076812076112075AD2AF22AE6EAF6FC298
:101D5000AF12075A12075A12075A12073FDEF21241
:101D6000076F12073FDFF8D2AF2291ED91E591E5C1
:101D7000756E01756F01757000B14B7C05AD581221
:101D8000074BC3ED955870F5C3E55894014009C35E
:101D9000E55894FF4032A1A6916112183591EDC229
:101DA000AF75EF1291E5DCD50570C3E57094035073
:101DB0000280C691E5056FE56E149000B193F808B6
:101DC000C3E56F98500280AE91E591E5056EC3E5DD
:101DD0006E94115002809C12107C121835C2AF759F
:041DE000EF1291E588
:00000001FF
